:0800000000008A150A16922F78
:0C3F24008301831687168312871AFC2F76
:023F3000A02FC0
:083F3800000000000000000081
:103F4000830183162430980040309900831290300A
:103F50009800EB27C13C031DFC2F313099008301F1
:103F60004B309900F801EB2703178F00FE00EB2779
:103F700003178D00EB27F900FA00FA0A1F308400BE
:103F8000EB27840A8000FA0BC02FF808031DE82FE6
:103F9000031720308400640000088C00840A0008A5
:103FA0008E00840A83168C137E1F8C170C155530D7
:103FB0008D00AA308D008C14000000008C18DE2FBC
:103FC0000C1183128D0A7E1FF903F90BCB2FAF2F33
:103FD0004E309900B22F83010B30FB00FC01FD0134
:103FE0008C1EF52F1A08F80708006400FD0BF02F4F
:0E3FF000FC0BEF2FFB0BEE2F831698139C2F6C
:02400E00323F3F
:00000001FF
